:100000002BC009C012C01BC01BC01BC01BC01BC023
:1000100020C020C020C00FB60F9251E0F52E65D150
:1000200050E45ABF0F900FBE18950FB60F9252E0D2
:10003000F52E5BD150E85ABF0F900FBE189518955A
:100040001895189518950FB60F926BD00F900FBE9C
:1000500018951895189518950FED0DBF00E008BB81
:1000600000E102BB00E007BB02E101BB442711270E
:10007000949A0CE04A95F1F71A95E1F70A95D1F7B1
:1000800094980CE04A95F1F71A95E1F70A95D1F7A3
:10009000949A0CE04A95F1F71A95E1F70A95D1F791
:1000A00094980CE04A95F1F71A95E1F70A95D1F783
:1000B000949A0AE005BF00E00BBF00E00ABF00E031
:1000C00009BF0AEC08BF00E003BF00E00FBD00E07D
:1000D0000EBD00E00DBD00E00CBD00E00BBD00E07A
:1000E0000ABD00E001BD08E90AB904E0859909E00C
:1000F00009B900E008B9B0E0A8E5D0E0C0E6F0E05A
:10010000E0E000E00993C03EE9F700E00093600002
:1001100000E00093610008E0602E00E00BBF7894DF
:10012000FFCF5CB1543619F458E0652EDDC054346D
:1001300019F459E0652ED8C0573439F457E4752EB8
:1001400050EC5ABF60EC6BBFCFC0513439F451E46E
:10015000752E50EC5ABF60E46BBFC6C0523439F400
:1001600052E4752E50EC5ABF60E86BBFBDC05D34E1
:1001700039F45DE4752E50EC5ABF60E86BBFB4C033
:10018000553439F455E4752E60E06BBF3FEF16D15E
:10019000ABC0563511F41CD1A7C0533521F436B38A
:1001A0000DD110D1A1C0503371F460E06BBF60E09D
:1001B000E62E6AE5A62E69E4B62E6CE3C62E68E448
:1001C000D62E00D191C0513371F460E06BBF61E075
:1001D000E62E6DE2A62E63E1B62E6EE1C62E64E237
:1001E000D62EF0D081C0523371F460E06BBF62E074
:1001F000E62E66E1A62E68E7B62E6FE0C62E62E117
:10020000D62EE0D071C0533371F460E06BBF63E071
:10021000E62E6BE0A62E6BE2B62E67E0C62E69E8EE
:10022000D62ED0D061C0543371F460E06BBF64E06F
:10023000E62E65E0A62E64E8B62E63E0C62E65ECD9
:10024000D62EC0D051C0553371F460E06BBF65E06D
:10025000E62E63E0A62E62EAB62E62E0C62E63E8C2
:10026000D62EB0D041C0563371F460E06BBF66E06B
:10027000E62E62E0A62E60EBB62E61E0C62E62EEA0
:10028000D62EA0D031C0573371F460E06BBF67E069
:10029000E62E61E0A62E6FEBB62E61E0C62E62E47C
:1002A000D62E90D021C0583371F460E06BBF68E067
:1002B000E62E61E0A62E67E4B62E60E0C62E61EF62
:1002C000D62E80D011C0593371F460E06BBF69E065
:1002D000E62E60E0A62E6EECB62E60E0C62E61EA39
:1002E000D62E70D001C071D0089550E05EBD50E0B0
:1002F0005DBD50E05CBDABBCBABC50EC58BF59E032
:100300005EBD88249924572D5D3499F451E05EBD7B
:100310006F2D88B787FD0CC0613019F480B382FF60
:10032000F8CF80B383FFF5CF3CB548D03DB546D07C
:1003300040C098E058B756FFFDCF8C98CBBCDABCD4
:1003400050E458BF80B3669576956F7782FD6068FC
:100350007F7783FD70688C9A9A9561F7562D593096
:1003600019F458B756FFFDCF862E972E50E05EBD8C
:10037000ABBCBABC50E458BF5F2D513061F4582D6E
:1003800052955F705068352F19D0582D5F705069A5
:10039000352F14D00EC0523061F4592D52955F7034
:1003A000506A352F0BD0592D5F70506B352F06D00A
:1003B00000C0829BFECF839BFECF08955D9BFECF46
:1003C0003CB908953DE0FADF08953FE3F7DF089573
:1003D00031E4F4DF36E7F2DF32E7F0DF30E2EEDF80
:1003E00032E5ECDF33E5EADF32E3E8DF33E3E6DF93
:1003F00032E3E4DF30E2E2DF36E5E0DF31E3DEDFA7
:100400003EE2DCDF30E3DADF35E3D8DF30E2D6DFAF
:100410002E2D203061F430E2D1DF30E2CFDF36E341
:10042000CDDF30E3CBDF30E3C9DFCCDF89C0213063
:1004300061F430E2C3DF31E3C1DF32E3BFDF30E339
:10044000BDDF30E3BBDFBEDF7BC0223061F430E2D2
:10045000B5DF32E3B3DF34E3B1DF30E3AFDF30E306
:10046000ADDFB0DF6DC0233061F430E2A7DF34E3ED
:10047000A5DF38E3A3DF30E3A1DF30E39FDFA2DFB6
:100480005FC0243061F430E299DF39E397DF36E36F
:1004900095DF30E393DF30E391DF94DF51C0253007
:1004A00061F431E38BDF34E389DF34E387DF30E36A
:1004B00085DF30E383DF86DF43C0263061F431E33C
:1004C0007DDF39E37BDF32E379DF30E377DF30E371
:1004D00075DF78DF35C0273061F432E36FDF38E352
:1004E0006DDF38E36BDF30E369DF30E367DF6ADF5E
:1004F00027C0283061F433E361DF38E35FDF34E3A2
:100500005DDF30E35BDF30E359DF5CDF19C02930AA
:1005100061F435E353DF37E351DF36E34FDF30E398
:100520004DDF30E34BDF4EDF0BC03FE347DF3FE300
:1005300045DF3FE343DF3FE341DF3FE33FDF42DFB0
:0205400008951C
:00000001FF
